:03F0000002F00813
:03F0610002F003B7
:05F0030012F0A480FEE4
:04F06400AA82AB834E
:05F068001ABAFF011BB4
:0EF06D00C3E49A74808BF063F08095F0500F2E
:04F07B007CB07D04E4
:05F07F001CBCFF011D97
:06F08400EC4D70F780DE88
:01F08A002263
:05F08B00C2A875E104BC
:0BF0900090DF3BE0FABA01F875E102E6
:09F09B0090DF3BE0FABA0DF82207
:07F0A40090FE00E0FAC2A893
:03F0AB0075E1020A
:0EF0AE0090DF3BE0FBBB0DF87B0090000AC03A
:0AF0BC0002C00312F064D003D0027A
:0EF0C600C3EB9A500F90DF3AE0FC74806CFBB5
:06F0D40090FE00F080EC4C
:03F0DA0075E104D9
:0EF0DD0090DF3BE0FBBB01F890DF0074AAF06F
:09F0EB0090DF0174AAF075E10345
:0EF0F40090DF3BE0FBBB13F8900014C002124B
:08F10200F064D002A502F0AB9D
:06F03700E478FFF6D8FDAD
:08F015007900E94400601B7A58
:05F01D000090F10E78E7
:03F02200007593E3
:0AF0250000E493F2A308B80002050E
:08F02F0093D9F4DAF27593FFA6
:08F03D007800E84400600A7944
:03F04500007593C0
:06F0480000E4F309D8FC0E
:08F04E007800E84400600C7931
:0BF0560000900000E4F0A3D8FCD9FA01
:03F0080075810708
:0AF00B0012F10AE582600302F0032F
:04F10A0075820022E8
:00000001FF
